:100000000DC025C061C023C022C021C020C01FC0B8
:1000100087C01DC000010517418BFF0011241FBEC2
:10002000CFE9CDBF10E0A0E6B0E0E6EBF3E002C020
:1000300005900D92A636B107D9F710E0A6E6B0E01C
:1000400001C01D92AF36B107E1F773D1B2C1D8CF6D
:1000500026EB33E003C0F9013197F1F70197D8F7A8
:10006000089596B393FB992790F981E098278091A2
:100070006900880F892B809369008F7090E0089544
:1000800080916700811115C0909168008091640093
:10009000890F809368008091680018161CF086E034
:1000A0008093680080916800873018F082E0809328
:1000B000680008958091680018162CF480916800FB
:1000C00081508093680008951895F894A89584B796
:1000D000877F84BF81B5886181BD11BC78941092FF
:1000E000660003C080E190E0B3DFBBDF892BD1F76E
:1000F0008BB780628BBF82E087BB85B7806285BF8C
:10010000889585B78F7D85BF8BB78F7D8BBFF89422
:10011000A89581B5886181BD80E481BD78940895FA
:100120001F920F920FB60F9211242F933F934F936C
:100130005F936F937F938F939F93AF93BF93EF934F
:10014000FF9380916800811104C010926A001092A0
:100150006B0087DF892BD1F110926A0010926D003D
:1001600010926C0010926E00809166008F3F19F023
:100170008F5F8093660080916600863161F48FEF17
:1001800080936B0080916800811103C086E38093A7
:10019000660076DFBDC08C3B91F48091670091E0F2
:1001A00089278093670080916700882319F0109257
:1001B0006800AEC08091650080936800A9C0853357
:1001C00009F0A6C085E180936600A2C08091670017
:1001D000882319F010926A0099C0809168008823E2
:1001E00071F080916A008F3F19F08F5F80936A00F1
:1001F00080916B008F3F19F08F5F80936B0080912F
:100200006600982F9150943108F580916800811113
:100210000AC080916500809368008FEF80936A0028
:1002200010926B0073C080916B00853140F4809117
:100230006800863020F486E08093680067C0809173
:100240006800809365001092680060C081115EC0F4
:1002500080916800863069F480916C0090916D0007
:10026000019690936D0080936C008A3F954108F051
:1002700021DF349B43C04091610040936000809136
:10028000620080936100309163003093620025B179
:100290002093630090E0840F911D830F911D820FC6
:1002A000911D9595879595958795209168002130AA
:1002B00019F422E730E002C02CE730E08217930700
:1002C00030F480916E008F5F80936E0013C01092A7
:1002D0006E008D39910528F083E087BBC09AC498E1
:1002E0000DC08F38910530F083E187BB88B3816101
:1002F00088BB04C082E187BBC49AC09880916E001D
:100300008C3B18F0D7DE10926E00369A1092660081
:10031000FF91EF91BF91AF919F918F917F916F91DD
:100320005F914F913F912F910F900FBE0F901F90B3
:10033000189517BA88E088BB85BB82E087BB83E24B
:100340008FBD81E083BF81E687B9A29A86EC86B92A
:10035000479A8FEF89BD83E090E07ADE19BC81E097
:1003600090E076DE85B7877E806185BFAEDEC0E037
:1003700020916800332727FD30958C2F90E02817B7
:100380003907B1F3E0916800FF27E7FDF095EC5ED7
:10039000FF4FE491E9BDC091680081E090E058DE34
:1003A000809168008111E4CF81E090E051DE8DDE24
:0603B000DFCFF894FFCF3F
:0603B600AAAAAAAA010296
:00000001FF
